:020000040000FA
:0A0000000000000005EF01F018D128
:0800180065D1096A086EFF0EB4
:100020000826092200D0D8A01200030E076EE60EA3
:1000300002D8F5D7076AFE0F066EE86A075AD8A0FD
:1000400012000000060600D0F8D70E500C6E1218F1
:10005000186E0D50D8A411503AE00D267E0E03E321
:100060000D5E03E336D00D5E31E310C00AF00FC021
:100070000BF00C8E128E106A0F6A0E6A180E176E35
:100080000C320B320A3206E31450102613500F22A2
:1000900012500E220E320F321032172EF1D70EBE32
:1000A00007D010360F360E360D5210E00D060C3408
:1000B00016E3103E14D00F3E12D00E3E10D0D88062
:1000C0000E320F3210320D3E0AD003D016840D6A64
:1000D00002D016820D68106A0F6A800E0E6E18AE7E
:1000E0000E9E105012000DC017F00E5010C00EF0F2
:1000F000106E103617321032166A1036173602E3B9
:100100001684167E06E11680176A106A0F6A0E6A58
:100110000BD0172803E0D880103206D0D8901032C8
:1001200002E1168201D0168616B604D016A20FD0B0
:1001300016B407D07F0E106EFF0E0F6E0E6E0D6E92
:1001400023D0800E106E01D0106A000EF6D716B0C4
:10015000FBD70D6A9F0E1760EBD77E0E1764F4D79E
:100160009E0E175C07E0D89010320F320E320D321F
:10017000172AF6D716A408D0D880000E0D560E56B2
:100180000F56105610AEE0D70D5012000F6A106ACD
:10019000189E0AD0189E10AE07D0D880000E0D56BB
:1001A0000E560F561056188E960E176E105209E006
:1001B000080E17260EC00DF00FC00EF010C00FF085
:1001C00011D00F520FE1080E175E0E5007E1080E16
:1001D000175E0D5002E1105010D00D6A0F6E0DC069
:1001E0000EF00D6A0FBE06D0D8900D360E360F36C3
:1001F0001706F8D718AE0F9E17500DC010F00D6EF1
:100200000F500EC00FF00E6E1200400E166E4F0E05
:10021000AF6E240EAC6E900EAB6E00010F0EC16E71
:10022000070EB46EC69AC00E926EE00E936EC00EAC
:10023000946E956AE80E966E6CD0F2A403D0F29498
:10024000817A11009EAA19D0060EAB1412E1E2CFFA
:1002500076F0E1CF75F0772A11EE00F07750E126C5
:10026000000EE222AECFE7FF76C0E2FF75C0E1FFED
:100270001100AE50AE50AB98AB8811007750785C4F
:1002800014E0782AEACF07F0E9CF06F001EE00F09B
:100290007850E926000EEA22EF50066E07C0EAFF0A
:1002A00006C0E9FFD880120004D0E868066ED8A026
:1002B00012001200776A786A9D8A9F8AF28EF28C09
:1002C00012009D9A01EE00F0010EF46EF36AF3063F
:1002D000000EF45AEE6AF450F310F9E1776A786A86
:1002E0009D8A1200F29EE0CF96FAD8CF97FAE8CF17
:1002F00098FAF28E0001A192F29E96CAE0FF97CA88
:10030000D8FF98CAE8FFF28E10009EA8FED7AD6E07
:100310001200939A8A8A0A0E80DE939A8A9A92969B
:10032000899696928D9293948A94959C8C9C94989D
:100330008B9894928B9295928C9292928992929AA7
:10034000899A93988A9893908A9095988C98959486
:100350008C9494968B969290899096908D9093968B
:100360008A96959E8C9E949A8B9A94908B90959059
:100370008C90929489949298899896948D94939263
:100380008A92959A8C9A95968C9694948B94796A85
:10039000456A466A446A00EE7AF01C0EEE68E82E62
:1003A000FDD7636A646A656A666A676A686A696AC9
:1003B000486A476A4A6A496A4C6A4B6A4E6A4D6A99
:1003C000506A4F6A526A516A546A536A566A556A49
:1003D000586A576A5A6A596A5C6A5B6A5E6A5D6AF9
:1003E000606A5F6A626A616A65DF6BDFCD6AF29498
:1003F000F28A870ED56EB16AA192A082D08EA292A7
:10040000B10EB16E99EC09F099EC0BF06E2AE86A26
:100410006EB2010F6FB0010806E16F706A2A000E1C
:100420006B226C226D222ADF196EEC0E195C06E33A
:10043000FE0E195C01E21B6ACEEF05F019AE38D052
:100440001B6A8B0E195C05E119C01BF01C681D6846
:100450002DD09B0E195C05E119C01BF01E681F68AA
:1004600025D0AB0E195C05E119C01BF0206821688E
:100470001DD0BB0E195C05E119C01BF02268236872
:1004800015D0CB0E195C04E119C01BF024680ED006
:10049000DB0E195C04E119C01BF0256807D0EB0ED8
:1004A000195C04E119C01BF026682768CCEF05F041
:1004B0001B5204E1CEEF05F0CCEF05F08B0E1B5C78
:1004C000D8A468D01C2803E119C01CF05FD019C063
:1004D0001DF06C0E1C5C0AE1449C469C79BC03D068
:1004E0008B968B9402D08C928C904DD06D0E1C5CB0
:1004F0000AE1449A469A79BA03D08C948C9602D039
:100500008B928B9040D06E0E1C5C0AE1449846980A
:1005100079B803D08C988C9A02D08B988B9A33D070
:100520006F0E1C5C0AE14496469679B603D08A9019
:100530008A9202D08C9C8C9E26D0700E1C5C0AE1A4
:100540004494469479B403D08A988D9402D08A94C6
:100550008A9619D0710E1C5C0AE14492469279B2D7
:1005600003D0899A899802D08D928D900CD0720E0A
:100570001C5C09E14490469079B003D0899289943B
:1005800002D0899689901C68CCEF05F0CEEF05F07B
:10059000CCEF05F09B0E1B5CD8A49BEF05F01E284A
:1005A00004E119C01EF099EF05F019C01FF01F52A9
:1005B000D8A461D06C0E1E5C0AE1449C469C79BCB8
:1005C00003D08B968B9402D08C928C9050D06D0E71
:1005D0001E5C0AE1449A469A79BA03D08C948C96B0
:1005E00002D08B928B9043D06E0E1E5C0AE1449831
:1005F000469879B803D08C988C9A02D08B988B9AB5
:1006000036D06F0E1E5C0AE14496469679B603D04A
:100610008A908A9202D08C9C8C9E29D0700E1E5C8F
:100620000AE14494469479B403D08A988D9402D018
:100630008A948A961CD0710E1E5C0AE144924692FE
:1006400079B203D0899A899802D08D928D900FD07B
:10065000720E1E5C0AE14490469079B003D08992F4
:10066000899402D08996899002D0CEEF05F0CCEF24
:1006700005F099EF05F06C0E1E5CD8A452D079BC41
:1006800003D08B948C8202D08C908B86797C448CA6
:1006900008EE96F0D8901F34E926000EEA22EECF3D
:1006A00061F0EFCF62F061506A24006E62506B20FF
:1006B000016E000E6C20026E000E6D20036E03C0F2
:1006C00095F002C094F001C093F000C092F069521E
:1006D00027E0468C09EE96F0D8906934E926000EA2
:1006E000EA22EECF00F0EFCF01F00050615C015044
:1006F000625805E362C054F061C053F011D009EEB6
:1007000096F0D8906934E926000EEA22EECF00F088
:10071000EFCF01F06150005C536E62500158546E8F
:1007200006D26D0E1E5CD8A452D079BA03D08C9636
:100730008B8202D08B908C84797A448A07EE96F073
:10074000D8901F34E926000EEA22EECF5FF0EFCFFB
:1007500060F05F506A24006E60506B20016E000EE6
:100760006C20026E000E6D20036E03C091F002C07B
:1007700090F001C08FF000C08EF0685227E0468AEA
:1007800009EE96F0D8906834E926000EEA22EECF02
:1007900000F0EFCF01F000505F5C0150605805E3BE
:1007A00060C052F05FC051F011D009EE96F0D890C1
:1007B0006834E926000EEA22EECF00F0EFCF01F018
:1007C0005F50005C516E60500158526EB0D16E0E99
:1007D0001E5CD8A452D079B803D08C9A8B8802D0F2
:1007E0008B9A8C887978448806EE96F0D8901F34DE
:1007F000E926000EEA22EECF5DF0EFCF5EF05D500D
:100800006A24006E5E506B20016E000E6C20026E3A
:10081000000E6D20036E03C08DF002C08CF001C08D
:100820008BF000C08AF0675227E0468809EE96F008
:10083000D8906734E926000EEA22EECF00F0EFCF21
:1008400001F000505D5C01505E5805E35EC050F061
:100850005DC04FF011D009EE96F0D8906734E926CC
:10086000000EEA22EECF00F0EFCF01F05D50005C09
:100870004F6E5E500158506E5AD16F0E1E5CD8A458
:1008800052D079B603D08A928C8C02D08C9E8A800A
:100890007976448605EE96F0D8901F34E926000E4E
:1008A000EA22EECF5BF0EFCF5CF05B506A24006E83
:1008B0005C506B20016E000E6C20026E000E6D20ED
:1008C000036E03C089F002C088F001C087F000C049
:1008D00086F0665227E0468609EE96F0D890663498
:1008E000E926000EEA22EECF00F0EFCF01F0005033
:1008F0005B5C01505C5805E35CC04EF05BC04DF0A2
:1009000011D009EE96F0D8906634E926000EEA225E
:10091000EECF00F0EFCF01F05B50005C4D6E5C500D
:1009200001584E6E04D1700E1E5CD8A452D079B41A
:1009300003D08D948A8402D08A968A8879744484FC
:1009400004EE96F0D8901F34E926000EEA22EECF8E
:1009500059F0EFCF5AF059506A24006E5A506B206C
:10096000016E000E6C20026E000E6D20036E03C03F
:1009700085F002C084F001C083F000C082F06552AF
:1009800027E0468409EE96F0D8906534E926000EFB
:10099000EA22EECF00F0EFCF01F00050595C015099
:1009A0005A5805E35AC04CF059C04BF011D009EE2B
:1009B00096F0D8906534E926000EEA22EECF00F0DA
:1009C000EFCF01F05950005C4B6E5A5001584C6EFD
:1009D000AED0710E1E5CD8A452D079B203D08998E3
:1009E0008D8202D08D90898A7972448203EE96F0CE
:1009F000D8901F34E926000EEA22EECF57F0EFCF51
:100A000058F057506A24006E58506B20016E000E4B
:100A10006C20026E000E6D20036E03C081F002C0D8
:100A200080F001C07FF000C07EF0645227E0468273
:100A300009EE96F0D8906434E926000EEA22EECF53
:100A400000F0EFCF01F00050575C0150585805E31B
:100A500058C04AF057C049F011D009EE96F0D8902E
:100A60006434E926000EEA22EECF00F0EFCF01F069
:100A70005750005C496E585001584A6E58D0720E5B
:100A80001E5CD8A452D079B003D08994898602D054
:100A9000899089827970448002EE96F0D8901F3454
:100AA000E926000EEA22EECF55F0EFCF56F0555072
:100AB0006A24006E56506B20016E000E6C20026E90
:100AC000000E6D20036E03C07DF002C07CF001C0FB
:100AD0007BF000C07AF0635227E0468009EE96F082
:100AE000D8906334E926000EEA22EECF00F0EFCF73
:100AF00001F00050555C0150565805E356C048F0CF
:100B000055C047F011D009EE96F0D8906334E9262D
:100B1000000EEA22EECF00F0EFCF01F05550005C5E
:100B2000476E56500158486E02D01E6837D01E6876
:100B300033D034D031D0AB0E1B5C0BE1202803E165
:100B400019C020F004D019C021F049EC08F026D0DB
:100B500023D0BB0E1B5C0BE1222803E119C022F05D
:100B600004D019C023F0F1EC08F018D015D0CB0E4A
:100B70001B5C08E1242804E119C024F0EBEC08F028
:100B80000DD00AD0DB0E1B5C07E1252804E119C05B
:100B900025F0EFEC08F002D00FEC08F0070E745CC3
:100BA000D8B007EF08F070506A5C71506B58725003
:100BB0006C5873506D58D8A01BD2738E060E745C9F
:100BC000D8A449D046BC0AD0449C8B948C908B9678
:100BD0008C9295699469936992693CD044AC1DD01C
:100BE00079BC03D08B968B8402D08C928C8053502E
:100BF0006A24006E54506B20016E000E6C20026E51
:100C0000000E6D20036E03C095F002C094F001C089
:100C100093F000C092F0449C1DD079BC03D08B941B
:100C20008C8202D08C908B86797C61506A24006E15
:100C300062506B20016E000E6C20026E000E6D2063
:100C4000036E03C095F002C094F001C093F000C0A1
:100C500092F0448CCCD1050E745CD8A449D046BA2D
:100C60000AD0449A8C968B908C948B92916990695F
:100C70008F698E693CD044AA1DD079BA03D08C9478
:100C80008C8602D08B928B8051506A24006E525019
:100C90006B20016E000E6C20026E000E6D20036E44
:100CA00003C091F002C090F001C08FF000C08EF040
:100CB000449A1DD079BA03D08C968B8202D08B9047
:100CC0008C84797A5F506A24006E60506B20016ECC
:100CD000000E6C20026E000E6D20036E03C091F0BA
:100CE00002C090F001C08FF000C08EF0448A7FD126
:100CF000040E745CD8A449D046B80AD044988C9AA3
:100D00008B9A8C988B988D698C698B698A693CD099
:100D100044A81DD079B803D08C988C8A02D08B98C7
:100D20008B8A4F506A24006E50506B20016E000E6B
:100D30006C20026E000E6D20036E03C08DF002C0A9
:100D40008CF001C08BF000C08AF044981DD079B8B7
:100D500003D08C9A8B8802D08B9A8C8879785D50DE
:100D60006A24006E5E506B20016E000E6C20026ED5
:100D7000000E6D20036E03C08DF002C08CF001C028
:100D80008BF000C08AF0448832D1030E745CD8A482
:100D900049D046B60AD044968A928C9E8A908C9C02
:100DA00089698869876986693CD044A61DD079B66F
:100DB00003D08A908A8202D08C9C8C8E4D506A24FB
:100DC000006E4E506B20016E000E6C20026E000E05
:100DD0006D20036E03C089F002C088F001C087F067
:100DE00000C086F044961DD079B603D08A928C8CD0
:100DF00002D08C9E8A8079765B506A24006E5C50AB
:100E00006B20016E000E6C20026E000E6D20036ED2
:100E100003C089F002C088F001C087F000C086F0EE
:100E20004486E5D0020E745CD8A449D046B40AD0FA
:100E300044948D948A968A988A9485698469836992
:100E400082693CD044A41DD079B403D08A988D84A3
:100E500002D08A948A864B506A24006E4C506B20D4
:100E6000016E000E6C20026E000E6D20036E03C03A
:100E700085F002C084F001C083F000C082F0449489
:100E80001DD079B403D08D948A8402D08A968A8842
:100E9000797459506A24006E5A506B20016E000E0E
:100EA0006C20026E000E6D20036E03C085F002C040
:100EB00084F001C083F000C082F0448498D0010E19
:100EC000745CD8A449D046B20AD0449289988D90D7
:100ED000899A8D92816980697F687E683CD044A23E
:100EE0001DD079B203D0899A898802D08D928D80E5
:100EF00049506A24006E4A506B20016E000E6C202F
:100F0000026E000E6D20036E03C081F002C080F0FF
:100F100001C07FF000C07EF044921DD079B203D0B2
:100F200089988D8202D08D90898A797257506A246F
:100F3000006E58506B20016E000E6C20026E000E89
:100F40006D20036E03C081F002C080F001C07FF00D
:100F500000C07EF044824BD07452D8A448D046B032
:100F60000AD0449089948990899289967D687C689A
:100F70007B687A683CD044A01DD079B003D08992B8
:100F8000898402D08996898047506A24006E48502F
:100F90006B20016E000E6C20026E000E6D20036E41
:100FA00003C07DF002C07CF001C07BF000C07AF08D
:100FB00044901DD079B003D08994898602D089905D
:100FC0008982797055506A24006E56506B20016EEC
:100FD000000E6C20026E000E6D20036E03C07DF0CB
:100FE00002C07CF001C07BF000C07AF0448017D8CA
:100FF0006DAE0CD06D6A6C6A6B6A6A6A446A466A46
:1010000000EE7AF01C0EEE68E82EFDD706D06DAE2D
:1010100004D06D6A6C6A6B6A6A6A06EF02F07468E3
:10102000738E1A6A070E1A5C33E2D8901A34E96E8E
:10103000EA6AEA36E936EA367A0EE926000EEA224C
:10104000EFCF00F0ECCF01F0ECCF02F0ECCF03F0EB
:101050007050005C71500158725002587350035820
:1010600015E2D8901A34E96EEA6AEA36E936EA36C9
:101070007A0EE926000EEA22EFCF70F0ECCF71F085
:10108000ECCF72F0ECCF73F01AC074F01A2ACAE3F6
:101090001200720E205C14E121C063F063520CE078
:1010A00009EE96F0D8906334E926000EEA22EECFDE
:1010B00047F0EFCF48F003D0486A476A469089D09E
:1010C000710E205C14E121C064F064520CE009EE62
:1010D00096F0D8906434E926000EEA22EECF49F06B
:1010E000EFCF4AF003D04A6A496A469272D0700E36
:1010F000205C14E121C065F065520CE009EE96F029
:10110000D8906534E926000EEA22EECF4BF0EFCFFF
:101110004CF003D04C6A4B6A46945BD06F0E205C57
:1011200014E121C066F066520CE009EE96F0D8900A
:101130006634E926000EEA22EECF4DF0EFCF4EF0F6
:1011400003D04E6A4D6A469644D06E0E205C14E180
:1011500021C067F067520CE009EE96F0D890673432
:10116000E926000EEA22EECF4FF0EFCF50F003D089
:10117000506A4F6A46982DD06D0E205C14E121C054
:1011800068F068520CE009EE96F0D8906834E926D1
:10119000000EEA22EECF51F0EFCF52F003D0526AA8
:1011A000516A469A16D06C0E205C13E121C069F09A
:1011B00069520CE009EE96F0D8906934E926000EE9
:1011C000EA22EECF53F0EFCF54F003D0546A536AC3
:1011D000469C2068120024681200266812002568C8
:1011E00012001E0E225CD8A475D0235217E1466A65
:1011F000486A476A636A4A6A496A646A4C6A4B6A1F
:10120000656A4E6A4D6A666A506A4F6A676A526AD0
:10121000516A686A546A536A696A5BD023C063F092
:1012200009EE96F0D8902334E926000EEA22EECF9C
:1012300047F0EFCF48F023C064F009EE96F0D89065
:101240002334E926000EEA22EECF49F0EFCF4AF030
:1012500023C065F009EE96F0D8902334E926000EFD
:10126000EA22EECF4BF0EFCF4CF023C066F009EE50
:1012700096F0D8902334E926000EEA22EECF4DF006
:10128000EFCF4EF023C067F009EE96F0D8902334EC
:10129000E926000EEA22EECF4FF0EFCF50F023C048
:1012A00068F009EE96F0D8902334E926000EEA2281
:1012B000EECF51F0EFCF52F023C069F009EE96F077
:1012C000D8902334E926000EEA22EECF53F0EFCF78
:1012D00054F00ED0420E225C07E1235203E1459008
:1012E00009D801D0458004D07B0E225CD8B402D846
:1012F00022681200446A466A89928996899A8D9278
:101300008A988A948A908C9C8C988B988C948B92D7
:101310008C928B96899089948D9089988A968D94D9
:101320008C9E8A928B9A8C9A8B908C968C908B94B4
:101330001200090197699669A20E996FC30E986F02
:101340009A0E9B6F460E9A6F960E9D6F320E9C6F93
:10135000920E9F6F3A0E9E6F8E0EA16F5D0EA06F64
:101360008A0EA36F9A0EA26F860EA56FF00EA46F61
:10137000830EA76F5F0EA66F7F0EA96FE70EA86F93
:101380007C0EAB6F850EAA6F790EAD6F3B0EAC6F06
:10139000760EAF6F070EAE6F720EB16FE80EB06FC4
:1013A0006F0EB36FDF0EB26F6C0EB56FEA0EB46FD7
:1013B0006A0EB76F0A0EB66F670EB96F3C0EB86F44
:1013C000640EBB6F820EBA6F610EBD6FDA0EBC6F1A
:1013D0005F0EBF6F440EBE6F5C0EC16FBF0EC06F5D
:1013E0005A0EC36F4C0EC26F570EC56FE90EC46F15
:1013F000550EC76F960EC66F530EC96FC86F510E4C
:10140000CB6F200ECA6F4E0ECD6FFB0ECC6F4C0E05
:10141000CF6FE50ECE6F4A0ED16FDC0ED06F480E47
:10142000D36FE20ED26F460ED56FF50ED46F450E18
:10143000D76F150ED66F430ED96F420ED86F410E7F
:10144000DB6F7B0EDA6F3F0EDD6FC00EDC6F3E0E82
:10145000DF6F100EDE6F3C0EE16F6D0EE06F3A0E27
:10146000E36FD40EE26F390EE56F460EE46F370E70
:10147000E76FC20EE66F360EE96F490EE86F340E65
:10148000EB6FDA0EEA6F330EED6F740EEC6F320E07
:10149000EF6F180EEE6F300EF16FC50EF06F2F0E5E
:1014A000F36F7B0EF26F2E0EF56F3A0EF46F2D0E6A
:1014B000F76F020EF66F2B0EF96FD10EF86F2A0E32
:1014C000FB6FA90EFA6F290EFD6F880EFC6F280EB8
:1014D000FF6F6F0EFE6F270E0A01016F5E0E006F29
:1014E000260E036F530E026F250E056F500E046F0C
:1014F000240E076F540E066F230E096F5E0E086FE1
:10150000220E0B6F6F0E0A6F210E0D6F860E0C6F81
:10151000200E0F6FA30E0E6F1F0E116FC60E106FF1
:101520001E0E136FEF0E126F1E0E156F146F1D0E31
:10153000176F520E166F1C0E196F8C0E186F1B0E44
:101540001B6FCB0E1A6F1B0E1D6F0F0E1C6F1A0E2A
:101550001F6F580E1E6F190E216FA50E206F180EEB
:10156000236FF80E226F180E256F4F0E246F170E83
:10157000276FAB0E266F170E296F0A0E286F160EF7
:101580002B6F6F0E2A6F150E2D6FD70E2C6F150E49
:101590002F6F430E2E6F140E316FB30E306F140E7B
:1015A000336F270E326F130E356F9F0E346F130E8D
:1015B000376F1A0E366F120E396F990E386F120E82
:1015C0003B6F1B0E3A6F110E3D6FA10E3C6F110E5B
:1015D0003F6F290E3E6F100E416FB50E406F100E1B
:1015E000436F440E426F0F0E456FD60E446F0F0EC1
:1015F000476F6B0E466F0F0E496F030E486F0E0E4E
:101600004B6F9D0E4A6F0E0E4D6F3A0E4C6F0D0EC6
:101610004F6FDA0E4E6F0D0E516F7C0E506F0D0E28
:10162000536F210E526F0C0E556FC80E546F0C0E77
:10163000576F720E566F0C0E596F1E0E586F0B0EB1
:101640005B6FCC0E5A6F0B0E5D6F7C0E5C6F0B0EDA
:101650005F6F2E0E5E6F0A0E616FE30E606F0A0EF3
:10166000636F990E626F0A0E656F510E646F0A0EFA
:10167000676F0B0E666F090E696FC80E686F090EF3
:101680006B6F850E6A6F090E6D6F450E6C6F090EDC
:101690006F6F060E6E6F080E716FC90E706F080EB9
:1016A000736F8E0E726F080E756F540E746F080E86
:1016B000776F1C0E766F070E796FE50E786F070E49
:1016C0007B6FAF0E7A6F070E7D6F7B0E7C6F070E00
:1016D0007F6F490E7E6F070E816F170E806F060EAB
:1016E000836FE70E826F060E856FB90E846F060E4C
:1016F000876F8B0E866F060E896F5F0E886F060EE2
:101700008B6F340E8A6F060E8D6F0A0E8C6F050E6E
:101710008F6FE10E8E6F050E916FB90E906F050EF3
:10172000936F930E926F050E956F6D0E946F00017F
:1017300012000201996B2F0E986F9B6B340E9A6FFB
:101740009D6B390E9C6F9F6B3E0E9E6FA16B420E80
:10175000A06FA36B470EA26FA56B4C0EA46FA76B77
:10176000510EA66FA96B560EA86FAB6B5B0EAA6FDE
:10177000AD6B600EAC6FAF6B650EAE6FB16B690E8B
:10178000B06FB36B6E0EB26FB56B730EB46FB76B99
:10179000780EB66FB96B7D0EB86FBB6B820EBA6FE9
:1017A000BD6B870EBC6FBF6B8C0EBE6FC16B900E96
:1017B000C06FC36B950EC26FC56B9A0EC46FC76BBB
:1017C0009F0EC66FC96BA40EC86FCB6BA90ECA6FF4
:1017D000CD6BAE0ECC6FCF6BB30ECE6FD16BB70EA1
:1017E000D06FD36BBC0ED26FD56BC10ED46FD76BDD
:1017F000C60ED66FD96BCB0ED86FDB6BD00EDA6FFF
:10180000DD6BD50EDC6FDF6BDA0EDE6FE16BDE0EAB
:10181000E06FE36BE30EE26FE56BE80EE46FE76BFE
:10182000ED0EE66FE96BF20EE86FEB6BF70EEA6F09
:10183000ED6BFC0EEC6F010EEF6FEE6FF16F050EAE
:10184000F06F010EF36F0A0EF26F010EF56F0F0EBF
:10185000F46F010EF76F140EF66F010EF96F190E8B
:10186000F86F010EFB6F1E0EFA6F010EFD6F230E57
:10187000FC6F010EFF6F280EFE6F010E0301016F5A
:101880002C0E006F010E036F310E026F010E056FFB
:10189000360E046F010E076F3B0E066F010E096FC7
:1018A000400E086F010E0B6F450E0A6F010E0D6F93
:1018B0004A0E0C6F010E0F6F4F0E0E6F010E116F5F
:1018C000530E106F010E136F580E126F010E156F2D
:1018D0005D0E146F010E176F620E166F010E196FF9
:1018E000670E186F010E1B6F6C0E1A6F010E1D6FC5
:1018F000710E1C6F010E1F6F760E1E6F010E216F91
:101900007A0E206F010E236F7F0E226F010E256F5E
:10191000840E246F010E276F890E266F010E296F2A
:101920008E0E286F010E2B6F930E2A6F010E2D6FF6
:10193000980E2C6F010E2F6F9D0E2E6F010E316FC2
:10194000A10E306F010E336FA60E326F010E356F90
:10195000AB0E346F010E376FB00E366F010E396F5C
:10196000B50E386F010E3B6FBA0E3A6F010E3D6F28
:10197000BF0E3C6F010E3F6FC40E3E6F010E416FF4
:10198000C80E406F010E436FCD0E426F010E456FC2
:10199000D20E446F010E476FD70E466F010E496F8E
:1019A000DC0E486F010E4B6FE10E4A6F010E4D6F5A
:1019B000E60E4C6F010E4F6FEB0E4E6F010E516F26
:1019C000EF0E506F010E536FF40E526F010E556FF4
:1019D000F90E546F010E576FFE0E566F020E596FBF
:1019E000030E586F020E5B6F080E5A6F020E5D6F8A
:1019F0000D0E5C6F020E5F6F120E5E6F020E616F56
:101A0000160E606F020E636F1B0E626F020E656F23
:101A1000200E646F020E676F250E666F020E696FEF
:101A20002A0E686F020E6B6F2F0E6A6F020E6D6FBB
:101A3000340E6C6F020E6F6F390E6E6F020E716F87
:101A40003D0E706F020E736F420E726F020E756F55
:101A5000470E746F020E776F4C0E766F020E796F21
:101A6000510E786F020E7B6F560E7A6F020E7D6FED
:101A70005B0E7C6F020E7F6F600E7E6F020E816FB9
:101A8000640E806F020E836F690E826F020E856F87
:101A90006E0E846F020E876F730E866F020E896F53
:101AA000780E886F020E8B6F7D0E8A6F020E8D6F1F
:101AB000820E8C6F020E8F6F870E8E6F020E916FEB
:101AC0008B0E906F020E936F900E926F020E956FB9
:101AD000950E946F010E1A6E0001800E1A5CD8B03C
:101AE000B1D002EE96F0D8901A34E926000EEA2220
:101AF000EECF04F0EFCF05F004C00DF005C00EF0FE
:101B0000C6EC00F0660E146E136E260E126E800E7A
:101B1000116E25EC00F073EC00F0006E0EC001F0C9
:101B200002EE96F0D8901A34E926000EEA2200C0A0
:101B3000EEFF01C0EFFF02EE96F0D8901A34E926CE
:101B4000000EEA22EECF00F0EFCF01F003EE96F0A8
:101B5000D8901A34E926000EEA2200C0EEFF01C038
:101B6000EFFF02EE96F0D8901A34E926000EEA2232
:101B7000EECF00F0EFCF01F004EE96F0D8901A34DB
:101B8000E926000EEA2200C0EEFF01C0EFFF02EEE0
:101B900096F0D8901A34E926000EEA22EECF00F033
:101BA000EFCF01F005EE96F0D8901A34E926000E3A
:101BB000EA2200C0EEFF01C0EFFF02EE96F0D890DF
:101BC0001A34E926000EEA22EECF00F0EFCF01F042
:101BD00006EE96F0D8901A34E926000EEA2200C0EC
:101BE000EEFF01C0EFFF02EE96F0D8901A34E9261E
:101BF000000EEA22EECF00F0EFCF01F007EE96F0F4
:101C0000D8901A34E926000EEA2200C0EEFF01C087
:101C1000EFFF02EE96F0D8901A34E926000EEA2281
:101C2000EECF00F0EFCF01F008EE96F0D8901A3426
:101C3000E926000EEA2200C0EEFF01C0EFFF1A2ADB
:081C4000D8A04AD71200FFD71B
:020000040030CA
:0300010006160ED2
:020005008580F4
:060008000FC00FE00F40E5
:00000001FF
